:020000040000FA
:100000000004040000000000041A0000081A0000A8
:100010000C1A0000101A0000141A00000C1B00003B
:100020000C1B00000C1B0000181A00001C1A00001A
:10003000201A0000241A00000C1B0000281A0000DF
:100040002C1A0000301A0000341A0000381A000080
:100050003C1A0000401A0000441A0000481A000030
:100060000C1B00000C1B00004C1A0000501A000072
:10007000541A0000581A00005C1A00000C1B000003
:10008000601A0000641A00000C1B0000681A0000CF
:100090006C1A0000701A0000741A0000781A000030
:1000A0007C1A0000801A0000841A0000881A0000E0
:1000B0000C1B00000C1B00000C1B00008C1A000025
:1000C000901A0000941A0000981A00009C1A000070
:1000D000A01A0000A41A0000A81A0000AC1A000020
:1000E0000C1B00000C1B00000C1B0000B01A0000D1
:1000F000B41A00000C1B00000C1B0000B81A000012
:10010000BC1A00000C1B00000C1B00000C1B0000A4
:100110000C1B00000C1B00000C1B00000C1B000043
:10012000C01A00000C1B00000C1B0000C41A0000C9
:10013000C81A0000CC1A00000C1B00000C1B0000A9
:100140000C1B00000C1B0000D01A00000C1B000050
:100150000C1B00000C1B00000C1B0000D41A00003C
:100160000C1B00000C1B00000C1B0000D81A000028
:10017000DC1A0000E01A0000E41A0000E81A00008F
:10018000EC1A0000F01A0000F41A0000F81A00003F
:10019000FC1A0000001B0000041B0000081B0000EC
:1001A0000C1B00000C1B00000C1B00000C1B0000B3
:1001B0000C1B00000C1B00000C1B00000C1B0000A3
:1001C0000C1B00000C1B00000C1B00000C1B000093
:1001D0000C1B00000C1B00000C1B00000C1B000083
:1001E0000C1B00000C1B00000C1B00000C1B000073
:1001F0000C1B00000C1B00000C1B00000C1B000063
:10020000FFFFFF00FFFFFF00C8040000C80400005C
:10021000C8040000C8040000C8040000C8040000AE
:10022000C8040000C8040000C8040000C80400009E
:10023000C8040000C8040000C8040000C80400008E
:10024000C8040000C8040000C8040000C80400007E
:10025000C8040000C8040000C8040000C80400006E
:10026000C8040000C8040000C8040000C80400005E
:10027000C8040000C8040000C8040000C80400004E
:10028000C8040000C8040000C8040000C80400003E
:10029000C8040000C8040000C8040000C80400002E
:1002A000C8040000C8040000C8040000C80400001E
:1002B000C8040000C8040000C8040000C80400000E
:1002C000C8040000C8040000C8040000C8040000FE
:1002D000C8040000C8040000C8040000C8040000EE
:1002E000C8040000C8040000C8040000C8040000DE
:1002F000C8040000C8040000C8040000C8040000CE
:10030000C8040000C8040000C8040000C8040000BD
:10031000C8040000C8040000C8040000C8040000AD
:10032000C8040000C8040000C8040000C80400009D
:10033000C8040000C8040000C8040000C80400008D
:10034000C8040000C8040000C8040000C80400007D
:10035000C8040000C8040000C8040000C80400006D
:10036000C8040000C8040000C8040000C80400005D
:10037000C8040000C8040000C8040000C80400004D
:10038000C8040000C8040000C8040000C80400003D
:10039000C8040000C8040000C8040000C80400002D
:1003A000C8040000C8040000C8040000C80400001D
:1003B000C8040000C8040000C8040000C80400000D
:1003C000C8040000C8040000C8040000C8040000FD
:1003D000C8040000C8040000C8040000C8040000ED
:1003E000C8040000C8040000C8040000C8040000DD
:1003F000C8040000C8040000C8040000C8040000CD
:100800000FA220000E7F24000E01880000000000CF
:10081000000020000000E000020032000001200083
:1008200020028800140007005B0007000000E000C1
:1008300003003A0080682100010020000200370018
:100840000000200001002000810F70000100320034
:1008500014000700000020000000E0000200320049
:100860000000020000000000DC1402000000000094
:100870000040DA000000FE004440A90040112000C2
:100880000000E0000300320000002000A00188000A
:100890004440A800000006008A1F78008B1F7800E3
:1008A0000000060091018800800478000000EB0041
:1008B0001A003700E284440032A0B4009905BA005F
:1008C000E284440032A0B4009906BA00E2844400F5
:1008D00032A0B4000006EB00476FDE00FD07B20057
:1008E000636CE10003003A00EBFF07000000EB003F
:1008F0000A003700606CE10004003A00005DEB0084
:100900008B05E900FDFF3E00040037006168E1004F
:10091000010032000086EB000B00070019C7BA0087
:100920001905BA000E04E00003003A000A00E000D6
:10093000E0FF3A0000000600FE07B2009E018800BA
:100940008A047800F5FF3700395DBA008B05E900AD
:100950000C003200295DBA008B05E9000800320066
:100960000C00E00003003A00E284440032A0B4002E
:10097000F5FF370019DDBA008B05E900FAFF3A00F0
:100980008904E800E184440032A0B40000000600BD
:100990000040DA000000FE00000005008001780041
:1009A00002003700815978000201E9000200E000EE
:1009B000FCFF3A00000006001201000000020000E7
:1009C0000000000000080000D80400003C00000007
:1009D0000001000001020000000100000902000007
:1009E000290000000101000000C0000032090000E1
:1009F00004000000000200000300000000000000EE
:100A0000092100001101000000010000221D00006A
:100A10000007000005810000034000000001000005
:100A20000705000001030000400000000100000075
:100A30000403000009040000340300004D0000001E
:100A40006900000063000000720000006F000000F9
:100A500063000000680000006900000070000000F2
:100A6000200000005400000065000000630000004A
:100A7000680000006E0000006F0000006C000000C5
:100A80006F000000670000007900000020000000F7
:100A9000490000006E000000630000002E0000000E
:100AA0002603000055000000530000004200000033
:100AB0002000000048000000490000004400000041
:100AC00020000000420000006F0000006F000000E6
:100AD000740000006C0000006F0000006100000066
:100AE00064000000650000007200000006000000C5
:100AF000FF09000001A10000011900000129000008
:100B00004015000000260000FF00000075080000EE
:100B100095400000810000001901000029400000FC
:100B200091000000C0000000EE8400001885000065
:100B30001C850000508500004572000061730000B4
:100B4000696E0000672000004465000076690000BF
:100B5000636500002E2E00002E000000457200008C
:100B60006173000065200000436F00006D7000009D
:100B70006C65000074650000005700007269000099
:100B800074650000204300006F6D0000706C000071
:100B900065740000650A0000507200006573000073
:100BA00073200000526500007365000074000000AF
:100BB000526500007365000074000000754D000070
:100BC0004F470000493200000A4200004F4F00002A
:100BD000544C00004F41000044450000520000000A
:100BE0000080FB008181FB00000140000281410088
:100BF0004311DD0003A020000301410012F0A10019
:100C00000104E00004003A0000004000A180200040
:100C1000823078000300370000004000E1802000AF
:100C20008230780012E0A1006401410012E0A000CF
:100C300000000600214A800080C0B300E78F50000A
:100C40000E003E0001407800818120009140780034
:100C50000104E00004003A0013C0B30082812000C8
:100C60000349780005003700E1CF500003003A0047
:100C700023C0B30082812000034978004194200002
:100C80000081FB00910811007140800080487800CD
:100C9000A1952000D1408800219420009100780087
:100CA000E1806000030032000004E0000C003A0024
:100CB000000006000004E000110032000294200051
:100CC00092017800D140800093587800D14088008C
:100CD0000309E8000040E900F8FF3A0000000600C0
:100CE0000294200092017800D1408000935878004F
:100CF000D14088000309E8000040E900F8FF3A000D
:100D00000000060000C8B30021952000914F10009C
:100D100033003A0001CCB300209420000148780051
:100D20005095200010407800E24F5000090032003A
:100D3000E34F500019003200E14F500026003A0006
:100D4000C04D2800004A880020012000204A880069
:100D500000000600409520001004E0000C003A005E
:100D60001080FB000000400041592800610078001D
:100D7000004A880041942000204190008248780079
:100D80008100E800304090008048780000000600B4
:100D9000209420000048EB00000006004095200051
:100DA00021C0B30090CF100008003E001080FB006F
:100DB000000040006159280061007800004A880066
:100DC0001080FB00204A88000000060020942000CC
:100DD0000048EB0000000600209420000048EB00D3
:100DE000000006000040EB00A1952000804878003C
:100DF0008100E800804878002095200010407800AD
:100E00007F4060000080FB00E10F50000B003200CB
:100E1000E20F50000C0032000000E00028003A0011
:100E2000209420001070A0000348E200240032004B
:100E30000100E9001014A0002100370020942000D8
:100E40001070A0001E003700209420001070A00039
:100E500060952000104078006F406000180032005C
:100E6000609520001004E000070035001040780075
:100E70006F4060000080FB0000004000A180200067
:100E8000E1007800070037006095200010407800EE
:100E90006F4060000080FB0000004000E180200007
:100EA000E10078000040280091006000808F500031
:100EB00003003A0011C0B300A0952000014878005B
:100EC000000820002194200011006000070032007B
:100ED000A0952000004A8800010078001000A000C2
:100EE00021C0B3000080E80001487800000006003F
:100EF000AA24AB0011003200A040800010419000F5
:100F000001C8B300814F51000B003A0071408000CE
:100F10001141900041C8B300814F510006003A00D2
:100F2000C1C0B30011409800A040800090409000E4
:100F30000174A00011409800AA24A9000008200014
:100F40005024880000000600881F78007040800050
:100F5000100478004E44DE00614464000020A200CA
:100F60007040880030408000E80F50000B003A00CD
:100F7000409520001080FB00F007B200B0248800EC
:100F80009604E20003003200000120003040880097
:100F900002003700400020003040880019C8BF0020
:100FA000E14F500021003A00A195200070408000E0
:100FB000110098001FFF070018C8BF00E24F500043
:100FC00008003A0041C0B300704080001140980012
:100FD00070408000904090000174A0001140980083
:100FE000200037000804E00008003A0081C4B30084
:100FF0007040800011409800704080009040900048
:101000000174A000114098001600370081C0B300A1
:101010007040800011409800704080009040900027
:101020000174A000114098000E0037008094200049
:101030001004E0000A003D00514A8000C808DE00AC
:10104000640040001080FB004800DD00008070005C
:101050000100320000000100809420001070A10007
:101060001968EF004F047800000006000468EF00E4
:101070000001EB008200780040072000ED0507002A
:101080008284A90000012000002488000968EF0084
:10109000000006008284A80000012000502488007F
:1010A00010C0B30004E8B7000968EF000001EB00CE
:1010B0008200780050072000DE053700889FBE00C0
:1010C0004095200011C0B30090CF10000E003A00F0
:1010D0000080E900104078007F4060000A003A007C
:1010E000209420001070A0003095200032C0B30082
:1010F000904F110003003A000140780003E8B70068
:10110000010037000368EF00409520001004E00064
:101110009C003A000080E900104078007F406000A9
:10112000E24F500097003A00609520001040780090
:101130006F406000930032006095200010407800FE
:101140006F4060000080FB00E10F50008D003C000C
:10115000000220000608E3008A003A0020942000E4
:101160001070A000609520001004E0000C00350015
:1011700010417800EF4061008180FB0081804000D9
:10118000A280200062847800104078006F406000E8
:101190000080FB0001952000E14478000C0037003E
:1011A0006095200010417800EF4061008180FB00D5
:1011B00081804000E2802000628478001040780046
:1011C0006F4060000080FB00E1942000E144780063
:1011D0000908A30002003A000820A100010037001E
:1011E0000820A000609520001004E00007003500F2
:1011F000104078006F4060000080FB00000040005D
:10120000A18020008830780007003700609520001A
:10121000104078006F4060000080FB00000040003C
:10122000E1802000883078003095200031C0B30084
:1012300090CF10001A003A001800E00013003D00A3
:10124000630040001004E000080035001040780002
:101250006F4060000080FB00019520006141780034
:101260000214A0008270780008003700609520000A
:10127000104078006F4060000080FB00E194200087
:10128000614178000214A0008270780098409000BC
:1012900040C8B30000C07000104498003900370007
:1012A000880078000120A2001100E00008003D0045
:1012B000114090000074A1000064A00090409800CC
:1012C00022002000500020005A05070003003700CC
:1012D000114090000064A000904098000918A300FD
:1012E00002003A001800E0001B003D00609520005D
:1012F0001004E00008003500104078006F406000E6
:101300000080FB0001952000614178000214A100DB
:101310008270780008003700609520001040780047
:101320006F4060000080FB00E19420006141780084
:101330000214A1008270780018409000B043B200FF
:1013400010449800220020008800780050002000FF
:10135000380507000300370018409000B043B20082
:101360001044980060952000104078006F406000A5
:101370000080FB0000004000A14A20000100400066
:101380001014A1004F04BE0000000600881F780062
:10139000209420001070A000AC24EF0008A02000D2
:1013A000020220008000EB00080078007BFD0700AF
:1013B0009424A8000040EB00E194200080487800CD
:1013C0000195200080487800F19420008048780042
:1013D00011952000804878001268EF009424A9003D
:1013E0006800440070408800A8408800B840880029
:1013F000409520001040780008E8B7000004E000A5
:1014000003003A0000012000304088000600370049
:1014100012002000818020000200780005050700EE
:1014200000022000304088004F04780000000600D1
:101430002095200001C6B30010C060003F003A00B4
:10144000309520001080FB008000EB00EB0F500077
:10145000E08F580039003E00006001001C0037009A
:101460001C003700350037001A0037003300370002
:10147000060037000A0037002C0037000A0037004A
:1014800008003700140037002000370020942000A7
:101490001070A0008000200030408800000006008E
:1014A00018FE3700B9FF370080802000004A88000E
:1014B000209420009000780013C0B3000081E80061
:1014C000034978001108B300010878000000060005
:1014D00044FE3700F9FE3700609520001081FB00C4
:1014E0002181200000942000010841000080E800D4
:1014F0009000780013C0B3000081E8000349780031
:101500001108B300010878000000060020942000B4
:101510001070A000609520009080FB0020812000CA
:101520004295200092707800000006000001EB0058
:101530008200780020002000BE04070000000600A2
:101540009EC0A9000080EB00702488005024880011
:10155000AA24EF00AC24EF002000200030258800F2
:10156000A824EF008644A900F00920008024880008
:101570006024880082C4A8008804A80000A020007D
:10158000C800DE00C12488000008EB00301078009D
:101590006000B8002050880031508800405088001A
:1015A0005150880060508800715088008050880039
:1015B00091508800A0508800B1508800C050880029
:1015C000D1508800E0508800F15088009424A80091
:1015D0009624EF0094A4A9009424A9008000200080
:1015E000502488008A64AB00FCFF3A000040EB0006
:1015F0002194200080487800819420000081FB0025
:10160000820878008180E80002F02F0091086100D4
:1016100013C0B30002822000034978001282200028
:10162000034978000268EF000068EF000468EF00EB
:101630000A28EF00E19420008048780001952000FE
:10164000804878001028EF000C28EF00F19420006B
:1016500080487800119520008048780080A0200004
:1016600070408800D0002000502588002095200080
:101670001050880081C0B30000A02000014878000D
:101680000000E80041C0B300014878001074A000D9
:101690000868EF002228EF002428EF000968EF0017
:1016A0000628EF0000000600889FBE008A1F780011
:1016B00000457800814478000984FB000838A300C5
:1016C000030032008040EB000A40780044FD070030
:1016D0000828A3000300320011C0B3000A407800BC
:1016E0003FFD07000A85FB000A054500A04A2000CF
:1016F00009707D004F0578004F04BE000000060011
:101700000104E000050032000082FB0004024200F8
:10171000E580200065027A00040037000082FB00AB
:1017200004024200A580200065027A008002EB00DE
:101730000400E0001A00320012029800034A780008
:10174000144190000244B2001242980014419000EB
:101750000234A00012429800144190000274A000CC
:10176000124298000104E000070032000080FB00F4
:1017700000004000E1802000008040001020A20016
:1017800084027800060037000080FB000000400063
:10179000A1802000008040001020A2008402780078
:1017A00005007800000006000004E00014003A0084
:1017B00081C0B300B040800001487800B040800094
:1017C0002195200011009800C1C0B300114098007D
:1017D000B0408000904090000174A000114098003B
:1017E00041C0B300704080001140980070408000FC
:1017F000904090000174A000114098000000060085
:101800008180FB000080FB00000040000080400061
:101810004300DD0002A0200082014000134290003E
:1018200041C8B30001427200944198006400400036
:10183000020040001041900081407100114098006A
:101840000000060094A4AB00190032000080FB00E9
:1018500000004000E18020000080400090007800FF
:101860001103BE00040420000500200006036200EE
:101870008003EB008688BE00900078001103BE0054
:1018800084186B0085906B00900078000120A20006
:1018900001087800914190000344B2009340980001
:1018A000100078009040900004C168001240980039
:1018B000000006002048E2002A003A0010C0B300F1
:1018C00020E8B7002148E20026003A0021E8B700EE
:1018D00019C8BF00E24F50000A003A007040800073
:1018E0000048EB0081C4B3007040800011409800B4
:1018F00070408000904090000174A000114098005A
:1019000000000600E14F500016003A001E68EF008C
:1019100080C0B300A140800080487800A2408000D1
:10192000219520001101980043C0B3001341980095
:10193000A2408000924190000374A00013419800DF
:1019400014C0B300E381200084497800B2408000D5
:1019500000497800B04080001100980001C8B30031
:101960001140980000000600A0408000104278005E
:10197000414A8000C808DE00A09420001080FB00CF
:101980004800DD00008070008480FB00808F5000E4
:1019900001003600004278008480FB000100500006
:1019A000819420004801DD00F30F20009181610047
:1019B000828871004800DE008180E800804878005D
:1019C0000404E000090032000000EB0061942000F4
:1019D00011017800A3952000634978008208E8008F
:1019E0000000E800804F5200F8FF3E00414A8000AE
:1019F000C808DE00A09420001080FB004800DD0035
:101A0000008070001900320081C0B300B040800037
:101A100001487800A1952000B04080001100980096
:101A2000A040800010E8A30008003A0081C4B30081
:101A3000B040800011409800B0408000904090007D
:101A40000174A000114098000000060081C0B3009E
:101A5000B040800011409800B0408000904090005D
:101A60000174A000114098000000060081C0B3007E
:101A7000B040800001487800B040800021952000EF
:101A80001100980041C0B30011409800B0408000A0
:101A9000904090000174A00011409800514A8000CD
:101AA000C808DE00C09420001080FB004800DD0064
:101AB00000807000010032000000010080942000CE
:101AC0001070A1000148E20001003A0079FF070010
:101AD0000000060019C8BF00E24F500001003A00A4
:101AE000A1FF37001968EF001E48E2000D003A0020
:101AF00081C0B300B040800001487800B040800051
:101B00002195200011009800C1C0B3001140980039
:101B1000B0408000904090000174A00011409800F7
:101B2000000006001E68EF00000006000268EF00DB
:101B30000068EF0019C8BF00E24F50000D003A00E6
:101B400081C0B300B040800001487800B040800000
:101B5000A19520001100980081C4B30011409800A5
:101B6000B0408000904090000174A00011409800A7
:101B700000000600809520001080FB009195200059
:101B80009180FB00C808DD008100700040942000B7
:101B9000908F500007003100809520009080FB005E
:101BA0000000E8001081FB004811DD004094200097
:101BB000010871001FFC0700A19520007040800003
:101BC0001100980081C4B30070408000114098005B
:101BD00070408000904090000174A0001140980077
:101BE0000000060094A4A900000820002194200011
:101BF000110060001F003A00809420001004E000F3
:101C000008003D0020C0B30019E8B7000048E2001A
:101C100001003A00C5FF07002168EF002068EF00CF
:101C20000000060081C0B300B04080000148780089
:101C3000B04080002195200011009800C1C0B30081
:101C400011409800B0408000904090000174A000C6
:101C50001140980041C0B3007040800011409800CE
:101C600070408000904090000174A00011409800E6
:101C700000000600209520001004E0000A003D004E
:101C800010C0B30019E8B7000248E20001003A00B2
:101C9000A6FF07002168EF002068EF000148E2007E
:101CA00014003A0003FF370020C0B30019E8B70062
:101CB00081C0B300B040800001487800B04080008F
:101CC000219520001100980041C0B30011409800F8
:101CD000B0408000904090000174A0001140980036
:101CE0002168EF002068EF000148E20001003A009F
:101CF000F0FE0700000006001868EF000168EF0022
:101D00000268EF000068EF001E68EF001968EF003E
:101D100070408000904090000174A1001140980034
:101D2000704080000020A200704088009040900029
:101D30000174A100114098000E48AA00B040800034
:101D4000904090000174A100114098002094200060
:101D50000048EB008000EB00214A880080942000BE
:101D60008180FB00010878000080E80001F02F006E
:101D700010886000AEFD07000001EB0082007800D3
:101D800030002000AB02070096FF3700D0C2B3003E
:101D90001FE8B700C1812000914078000100780061
:101DA000B00FB20013003A00C10FB20000A0200033
:101DB00080804000A1408800010078000020A2003F
:101DC000B040880002C023001101610000402300E0
:101DD000800F510006003A0011009000219520006C
:101DE00007000900B05878008000B100C2FF37003A
:101DF00038FF3700E80F500001003A0052FC07009E
:101E00000000060010418000214180006100400078
:101E1000E080480010418800214188000448E20029
:101E200004003A000948EC0009E8B70001003A0054
:101E300009E8EF0000000600881F780030408000AD
:101E40000000E00012003A009424EF008C24EF0020
:101E50002000200030258800A824EF008644A90037
:101E6000F0092000802488006024880082C4A80033
:101E70009404AB0003003A009404A8009404AB005F
:101E8000FDFF3200100020003040880002003700C3
:101E9000E10F500008003A0094C4AB0006003A007D
:101EA0008AA4EF008C24EF008C04A8008C84A80086
:101EB00020002000304088008084AB000500320004
:101EC0008284AB000300320000012000002488005F
:101ED00066FC07008824AB00020032008EC0A90017
:101EE000690037008A04AB00070032008C04AB00A5
:101EF0000500320092FD07004000200030408800BD
:101F000010002000502488008A84AB0003003200B7
:101F10008C84AB00010032005EFC070080C4AB0083
:101F2000030032000004200000248800B5FF0700F1
:101F30008A44AB000E0032008C44AB000400320037
:101F4000120020008000EB0030072000390207005B
:101F500040002000502488001FC8BF00030032004A
:101F60000040E9001FE8B70001003A0051FE0700F9
:101F70008AE4AB00030032008CE4AB0001003200C5
:101F8000DBFB07008A24AB00090032008C24AB0085
:101F900007003200120020008000EB00F0FF270055
:101FA000240207008EA4EF002000200050248800A7
:101FB00030408000E30F500002003E008EC0A900B8
:101FC000310037008C64AB002E00320048C0B300F3
:101FD0008A64AB0003003A002A0037008A64AB0031
:101FE0002800320091248000C08120000148780040
:101FF0000181FB004411DE000240780002427800BB
:10200000D381200084497800820020005224880077
:102010000138A30009003A008080FB0002952000EF
:10202000E2C1780061C261000404A2000304A100BF
:1020300084C1710003F17800080037008080FB0044
:10204000E2942000E2C1780061C261000404A200B1
:102050000304A10084C1710003F178000004E000D2
:1020600002003A0049FF0700040037000001EB00BE
:10207000C181200020072000EE0107000844E9008C
:10208000D6FF3A008EC0A9004F0478000000060079
:10209000104180002141800000000600881F780068
:1020A0002628EF002828EF0090CAB3002AE8B700DE
:1020B00000802A00604188002000200070418800D4
:1020C00018C0B30008407800818320008848780059
:1020D0003068EF0034A8EF0036A8EF003268EF0058
:1020E000D1C1B30070FD070003C4B300028C20000F
:1020F0008040EB000840780081FD070030418800F7
:102100004F0478000000060012832000124178007E
:102110000281FB008001EB004A18DD00C610DE00E2
:10212000810070004A10DD0022042400023B880078
:102130008141780022032000034978000081EB00F0
:102140000208BB001000FC0050052000303B880056
:10215000A00A2000303B880061E7A80000000000D2
:10216000000000006007E200FEFF350000000600EE
:1021700030002400003B880032C8BF001D00320040
:10218000019020000081FB008001EB00A441800051
:10219000B54180000201520083815A000342780059
:1021A0002003200004487800020078001108BB00DA
:1021B000110190000288BB001000FC0050052000B7
:1021C000303B8800A00A2000303B880061E7A8006F
:1021D00000000000000000006007E200FEFF350084
:1021E00032C8ED0032E8B700E48040000004E000AF
:1021F000E4FF3A0061C7A9000000060023032000A5
:1022000093417800400ADE00050020000443780076
:102210002203200006497800000178001282BA00EB
:10222000840078001200BA000342780022032000E4
:102230000449780000000600889FBE008A9FBE0007
:102240003048E20022003A00404180000000E000F7
:10225000020032001000E0007301350030418000C0
:102260000000E00005003A00F08B2000F183200020
:102270000204200000014100030037001000E000CC
:10228000F9FF3D0068013700D0687800820F5000E8
:10229000FDFF3A0003C4B300028C20008040EB0035
:1022A00010C0B30016FD07003041880010C0B30015
:1022B00030E8B700F0872000010420008080400053
:1022C0000068EB00810F5000FDFF3A005601370017
:1022D0000084200010407800E54F5000910032004B
:1022E00006003E00E34F50005A0032006E003E00F0
:1022F000E24F50004C013A0006003700E74F500013
:10230000E6003200DB003900E84F500046013A0099
:102310003A01370020C0B3000188200080487800CF
:1023200082C3B3008100E800824878008100E800A1
:102330008048780011C0B300308820000148780040
:102340000040EB00418820008048780082C1B30043
:102350008100E800824878008100E8008048780029
:102360008100E8008048780000802E00F1FF2F00F7
:102370006241800073418000020040008380480079
:10238000F20F200083882000824960004802DE00AE
:102390008301E800844978008301E80082C9600075
:1023A000C808DE000300E800014878000000E800EB
:1023B00000C8EB003848E20019003A0031C0B30011
:1023C000014878000040EB0082CFB300E380410079
:1023D00082487800B2CAB3008100E80082487800E1
:1023E00022C0B3008100E800824878008100E80044
:1023F0008048780082C0B3008100E80082487800FD
:102400008100E800804878008100E800804878007A
:102410008100E800804878000100E80000C8EB0077
:10242000404180000000E000020032001000E000A7
:10243000FD00350003C4B3000288200011C0B300C2
:1024400001407800AEFC0700404188003068EF0092
:10245000F5003700108420001004E00008003A0066
:10246000A0CAB3002AE8B70083BF2A0063418800EE
:1024700023002000734188003868EF00080037000F
:1024800090CAB3002AE8B70000802A0060418800A3
:10249000200020007041880010C0B30038E8B70069
:1024A0003068EF00E00037008000EB0010002000F3
:1024B00010010700C05928005601070060C0B30092
:1024C00031E8B7002AC8BF000080FB000000E80028
:1024D000E60F50000B0034000BFF070056FE07000C
:1024E0003148EC0031E8B7000080FB00A1822000F9
:1024F000914078008180FB008100E800810F50004E
:10250000F5FF350061C7A9003068EF008000EB00DF
:1025100010002000F7000700E05A28003D010700E6
:10252000C1003700A0418000B1418000E10F4000B0
:10253000E08F48000E003A00128420001281FB0058
:10254000238420009381FB00C819DD000300710083
:10255000328420001281FB00438420009381FB0021
:10256000C819DD0083007100A0418800B1418800D6
:10257000128420001281FB00238420009381FB0041
:10258000C819DD0003007100328420001281FB00B5
:10259000438420009381FB00C819DD008300710093
:1025A000A2418000B3418000820F5000838F580009
:1025B0002E003A005084200010407800E14F500077
:1025C0002A0036000044EB0021832000914078006F
:1025D0000181FB00820141000080FB00820320009A
:1025E000000051004F01DE00000041000081D100D9
:1025F0000880FB0000004100640040000000400033
:1026000002842000624278000482FB000000410046
:10261000104190004811DD0002017200009020007E
:1026200002B079000140E80032E8B700A241800022
:10263000B341800061014100E0814900A24188006E
:10264000B3418800FC4F500001003A00C8FE07006B
:102650000844E80050842000104078008080FB008F
:102660008100D100814F5400D7FF39003068EF005E
:102670006D003700BEFE070034A8EF0036A8EF005B
:102680003068EF008000EB00100020009900070088
:10269000D05B2800DF000700630037004041800066
:1026A0000000E000020032001000E0005E00350093
:1026B00071C0B30000882000014878001284200017
:1026C0001281FB00238420009381FB00C819DD00E8
:1026D00003007100328420001281FB00438420003B
:1026E0009381FB00C819DD0083007100F20F200008
:1026F00013882000824960004802DE008301E80060
:10270000844978008301E80082C96000C808DE00BF
:102710000300E80001487800508420001040780051
:102720008380E80080487800E14F50002B0036009D
:102730000044EB000881FB008001EB0014842000C2
:102740001482FB00258420009582FB00C82ADD004E
:1027500005007200348420001482FB0045842000B0
:102760009582FB00C82ADD0085007200020040004F
:1027700083804800A1FE07008884FB005484200069
:102780009482FB008502D1008583FB0007855400FD
:102790000A02B000068820000A0545000A05430029
:1027A000F40F2000044D6000C805DE001B459800B2
:1027B00081016200078054001002B0000000400058
:1027C0000000430004C86100C818DE0011409800F2
:1027D00008C4E80088CF5200D6FF3E0003C4B3000F
:1027E0000288200011C0B30001407800C4FB07003C
:1027F000404188003068EF000B0037008000EB009C
:10280000100020003B000700805D280081000700C9
:102810009424EF000080EB00000000000000E900BD
:10282000FDFF3A000000FE004F05BE004F04BE0051
:102830000000060031072000810F50000D0032001B
:1028400005003C00E10F500010003200E30F500083
:1028500011003A000F00370041072000810F50009F
:10286000080032008100E800810F50000A003A00A1
:1028700002003700FE00070007003700FC000700D9
:1028800005003700FA0007000300370003FE0700C9
:10289000010037007100070010000500EC22A800BD
:1028A000000000000000000000000000EC22A90071
:1028B0000000060000F02F00E022B600F002A900A0
:1028C000F022A900E822A900F402A900F422A9003C
:1028D000EC22A900000006000000FB0001F02F0020
:1028E000221780008280600080807000211788009D
:1028F0000000060080417800F00F2000E022B700C1
:10290000F422A800F402A900EC22A80000000000B4
:10291000000000000000000012178000EC22A90057
:102920000278A300F8FF3A0002F02F00002E2000EA
:1029300010086100F422A9008180FB008100EA00F8
:10294000CF08DE00A21780000200A1000281700003
:10295000A217880003407800DFFF0700CFFF370091
:10296000D4FF070000202100A10720001801070064
:102970008040EB0080C3B300DEFF07008040EB0027
:1029800080C0B300DBFF07008040EB0010C0B30045
:10299000D8FF07008040EB0060C0B300D5FF070000
:1029A0008040EB00C0C0B300D2FF070000B82B008E
:1029B0000100200006013700F0F32F004427B60085
:1029C00042A7AB0003003A000000000042A7AB00A2
:1029D000FDFF320040A7A900F0C2A900D022A80044
:1029E000DFFF07000000EB00E3000700D4FA070058
:1029F0000060FE0010FD070030408000FF0F500017
:102A0000FBFF36008824AB00F9FF3A000AFE0700FE
:102A1000F7FF3700881F780000047800184078001E
:102A20000004E0000B003200EA4F500004003A00BE
:102A30008040EB0000CCB300AEFF0700020037007F
:102A400011C0B300ABFF0700584078000004E0005D
:102A5000F5FF3A004F0478000000060020952000A2
:102A6000104078007F406000E14F500054003A0071
:102A7000609520001004E00051003A00630050000F
:102A800061C0B30090CF10001B003A000080E80046
:102A900010407800FBC04000814F5000040032001D
:102AA0008140E800814F500013003A000B003700CE
:102AB00008C8BF00E14F50000F003A000050280046
:102AC000004A880090002000204A880001CCB30012
:102AD0002094200001487800070037006057280044
:102AE000004A8800D0012000204A880001CCB300B1
:102AF00020942000014878002095200002C6B300F1
:102B00009040610000C2B30080CF50002C003A001A
:102B10003095200010407800E34F5000190032003B
:102B200003003E00E24F500025003A000500370048
:102B3000EA4F50000B003200EB4F500020003A00EB
:102B400018003700A0832000004A880010002000F1
:102B5000204A880011CCB30020942000014878005E
:102B60000000060001C8B30020942000014878004E
:102B70005095200010417800A18320008248780001
:102B800000000600B0832000004A880010002000EA
:102B9000204A880011C8B300209420000148780022
:102BA0000000060001C8B30020942000014878000E
:102BB0004095200010417800B183200082487800C1
:102BC00000000600E10F500003003200E20F500049
:102BD00004003A0002003700F4C2A800000006001A
:102BE000F4E2A80000000600E10F500003003200EC
:102BF000E20F500004003A0002003700F4C2A900BE
:102C000000000600F4E2A90000000600E10F5000F9
:102C100003003200E20F50000B003A0005003700BD
:102C200000042000F402B6000000EA004F00DE00BD
:102C30000000060000082000F402B6000000EA00D0
:102C40004F00DE000000060000000500E10F50000C
:102C500003003200E20F500004003A000200370087
:102C6000F0C2A90000000600F0E2A9000000060082
:102C70008824AB000200320010002000DAFF370089
:102C8000000220000608E30010003A00F041800036
:102C9000E10F500002003A00CAFF07001A00370097
:102CA000B1042000810F500003003A001000200002
:102CB000CDFF07001400370061092000810F50008C
:102CC000110036003E28EF000F003700F041800071
:102CD000E10F500002003A00BAFF07000A00370077
:102CE00021032000810F500003003A001000200053
:102CF000BDFF070004003700613B2000810F50003A
:102D0000010036003E28EF003E28EC0000000600DF
:102D10004009000022000000000000000008000040
:102D20002600000000000000000A00002000000053
:102D3000000000003A08000002000000000000004F
:102D4000400800000001000000000000260800000C
:102D500014000000000000003C0800000200000019
:102D600002000000010000003E0800000200000018
:102D700000000000000000000000E00013003A0026
:102D800083E0A800100020002700070010002000AA
:102D90001D0007000004E00006003A003008200093
:102DA0004007B6000300320083E0A900001A0400C7
:102DB00000000000E05D280016FF07001000200062
:102DC000A2FF070020002000A0FF0700000006006F
:102DD000F03FB1000180B10006003500EE030900AC
:102DE00000000000403FB1000180B100FBFF3D004A
:102DF0001000B000203FB000020035000080090044
:102E00000000000000000600E10F500005003A003D
:102E100090168000620060000000E9004F00DE00B4
:102E20000000060000000500E10F500001003A001C
:102E3000D022A80000000600FFFFFF00FFFFFF00F8
:10340000101B040000000000FC1B04000000000072
:10341000FC1B040000000000FC1B04000000000076
:10342000FC1B040000000000FC1B04000000000066
:10343000FC1B040000000000FC1B04000000000056
:10344000FC1B040000000000FC1B04000000000046
:10345000FC1B040000000000FC1B04000000000036
:10346000FC1B040000000000FC1B04000000000026
:10347000FC1B040000000000FC1B04000000000016
:10348000FC1B040000000000FC1B04000000000006
:10349000FC1B040000000000FC1B040000000000F6
:1034A000FC1B040000000000FC1B040000000000E6
:1034B000FC1B040000000000FC1B040000000000D6
:1034C000FC1B040000000000FC1B040000000000C6
:1034D000FC1B040000000000FC1B040000000000B6
:1034E000FC1B040000000000FC1B040000000000A6
:1034F000FC1B040000000000FC1B04000000000096
:10350000FC1B040000000000FC1B04000000000085
:10351000FC1B040000000000FC1B04000000000075
:10352000FC1B040000000000FC1B04000000000065
:10353000FC1B040000000000FC1B04000000000055
:10354000FC1B040000000000FC1B04000000000045
:10355000FC1B040000000000FC1B04000000000035
:10356000FC1B040000000000FC1B04000000000025
:10357000FC1B040000000000FC1B04000000000015
:10358000FC1B040000000000FC1B04000000000005
:10359000FC1B040000000000FC1B040000000000F5
:1035A000FC1B040000000000FC1B040000000000E5
:1035B000FC1B040000000000FC1B040000000000D5
:1035C000FC1B040000000000FC1B040000000000C5
:1035D000FC1B040000000000D81B040000000000D9
:1035E000FC1B040000000000FC1B040000000000A5
:1035F000FC1B040000000000FC1B04000000000095
:10360000FC1B040000000000FC1B04000000000084
:10361000FC1B040000000000FC1B04000000000074
:103620000FA220000E7F24000E0188000000000081
:10363000000020000000E000020032000001200035
:1036400020028800140007006D0007000000E00061
:1036500003003A00E07C2300010020000200370054
:103660000000200001002000810F700001003200E6
:1036700014000700000020000000E00002003200FB
:1036800000000200000000003838020000000000C6
:103690000040DA000000FE004440A900800F200036
:1036A0000000E0000300320000002000A0018800BC
:1036B0004440A800000006008A1F78008B1F780095
:1036C0000000060091018800800478000000EB00F3
:1036D0001A003700E284440032A0B4009905BA0011
:1036E000E284440032A0B4009906BA00E2844400A7
:1036F00032A0B4000006EB00476FDE00FD07B20009
:10370000636CE10003003A00EBFF07000000EB00F0
:103710000A003700606CE10004003A00005DEB0035
:103720008B05E900FDFF3E00040037006168E10001
:10373000010032000086EB000B00070019C7BA0039
:103740001905BA000E04E00003003A000A00E00088
:10375000E0FF3A0000000600FE07B2009E0188006C
:103760008A047800F5FF3700395DBA008B05E9005F
:103770000C003200295DBA008B05E9000800320018
:103780000C00E00003003A00E284440032A0B400E0
:10379000F5FF370019DDBA008B05E900FAFF3A00A2
:1037A0008904E800E184440032A0B400000006006F
:1037B0003600F800809FBE00829FBE00849FBE003E
:1037C000869FBE003400F80000002000A0018800A1
:1037D0000000FA000F0107000080FA003400F90031
:1037E0004F03BE004F02BE004F01BE004F00BE009F
:1037F0003600F900004006000040DA000000FE003C
:10380000000005008001780002003700B1597800FF
:103810000201E9000200E000FCFF3A00000006009F
:103820008001780002003700815978000201E90028
:103830000200E000FCFF3A00000006001201000058
:10384000000200000000000000080000D804000092
:103850003F00000000010000010200000001000024
:1038600009020000290000000101000000C0000062
:103870003209000004000000000200000300000004
:1038800000000000092100001101000000010000FB
:10389000221D000000070000058100000340000019
:1038A00000010000070500000103000040000000C7
:1038B0000100000004030000090400000A030000E6
:1038C0004D0000004F0000004700000049000000CC
:1038D00020030000750000004D0000004F000000B4
:1038E00047000000490000003200000020000000F6
:1038F00048000000490000004400000020000000D3
:1039000044000000650000006D0000006F00000032
:1039100006000000FF09000001A1000001190000DD
:10392000012900004015000000260000FF000000F3
:10393000750800009540000081000000190100009A
:103940002940000091000000C0000000309C0000F1
:103950005A9C00005E9C0000689C0000020400006D
:103960000E0100000F1100000F0000000204000013
:103970000E1100001F1000000E00000002040000E5
:103980000C040000040400000E000000020400000B
:103990000E110000111100000E00000002040000D2
:1039A00011110000111300000D0000000A000000BA
:1039B00011110000111300000D000000050A0000A5
:1039C00011110000111300000D000000050A000095
:1039D0000E110000111100000E000000040A00008A
:1039E0000A0A0000111F00000E000000000E000077
:1039F00015170000110E0000000000001C0200005E
:103A000001050000091E000008040000754D0000BB
:103A10004F470000493200002048000049440000A0
:103A200020440000656D00006F0000000200FA00F5
:103A30009EC0A9000080EB00702488000080EB008D
:103A400050248800AA24EF00220020008000EB0010
:103A5000C04A200072FF07002000200030258800A7
:103A6000A824EF008644A900F009200080248800E3
:103A7000F00920006024880082C4A8008804A800FF
:103A800000A020004800DE00C02488000040EB00B9
:103A9000004F7800070037001E80FB00C200DD00E9
:103AA00000A02000008140006000B8000089BE0036
:103AB0001E4FE8001E407800E74F5000F6FF36002A
:103AC0009424A8009624EF0094A4A9009424A900AB
:103AD0008000200050248800A08B20008040EB0054
:103AE00001487800008C20008040EB0001487800FD
:103AF00001468000F00F2000008060000046880032
:103B00001146800000F02F00008060001046880001
:103B100050248000680060000000E000ECFF3A00E4
:103B200010C0B3001BE8B70010C0B3001CE8B7001A
:103B30001D68EF001E68EF001568EF000040EB0005
:103B4000004F7800170037001E80FB008000400007
:103B5000C0802000008040008000EB000108780059
:103B60001E80FB008000400080802000008040001C
:103B70008000EB00010878009E80FB00608C200034
:103B8000008040008040EB00014878009E80FB00F0
:103B9000808C2000008040008040EB0001487800CD
:103BA0001E4FE8001E407800E14F5000E6FF36004F
:103BB00080A0200060408800D000200050258800B0
:103BC000A08C20001050880000A0200081C0B3000D
:103BD0000148780010A0200041C0B30001487800DF
:103BE00010A0200010407800804078000174A000F0
:103BF00010A02000014878000268EF002028EF00A4
:103C00002228EF002468EF000028EF000080FA006F
:103C1000000006000200FA0000408000E10F5000A2
:103C20000B003A00A1248000000420000080600006
:103C30000000E00006003A000080EB0050248800FD
:103C40008C04A8008C84A80020002000004088007C
:103C500000248000700060000000E00007003200D7
:103C600010248000700060000000E00003003200BB
:103C70000001200000248800BD04070040248000CB
:103C8000620060000000E000020032008EC0A90067
:103C9000A100370050248000610060000000E000B7
:103CA0000A00320060248000610060000000E00033
:103CB000060032005DFF07009EC0A8004000200003
:103CC000004088001000200050248800502480000C
:103CD000700060000000E0000500320060248000F9
:103CE000700060000000E000010032009304070053
:103CF0000124800000042000008060000000E0003B
:103D0000030032000004200000248800F3060700AE
:103D100050248000640060000000E00014003200C5
:103D200060248000640060000000E00004003200B5
:103D3000120020008000EB0030072000640C070018
:103D4000400020005024880019C8BF000004E00093
:103D50000300320019C8BF000040E90019E8B700AD
:103D600019C8BF000004E00001003A00A3010700E9
:103D70005124800000082000008060000000E00066
:103D800006003200612480000008200000806000EE
:103D90000000E000010032004C04070050248000C5
:103DA000620060000000E0000C003200602480002F
:103DB000620060000000E0000800320012002000F5
:103DC0008000EB00F0FF2700410C07000080EB00B3
:103DD00070248800200020005024880000408000CB
:103DE000E30F500002003E008EC0A9004A003700D9
:103DF00060248000680060000000E00045003200A0
:103E00000040EB00004F78003D0037005024800058
:103E1000680060000000E0003D0032009024800057
:103E20000040780016E8B70016C8BF000080FB000D
:103E30004400DE000040780017E8B7008000200052
:103E40005024880016C8BF00684060000004E000ED
:103E500011003A0017C8BF000081FB008080FB0002
:103E6000808C2000008040009040780061C060009D
:103E70000004A200E1406000808C200000004100AE
:103E8000E1C06000104178000204A100814071008F
:103E9000014878001000370017C8BF000081FB0000
:103EA0008080FB00608C2000008040009040780003
:103EB00061C060000004A200E1406000608C20004E
:103EC00000004100E1C06000104178000204A10040
:103ED000814071000148780017C8BF000004E0006D
:103EE00002003A002E040700040037000001EB0036
:103EF0006181200020072000F50B07001E4FE8001D
:103F00001E407800E34F5000C0FF3600010037002C
:103F1000000000008EC0A9000080FA00000006002A
:103F20000400FA0020479800314798003E40900076
:103F30000080FB00680060000000E0000300320029
:103F40008040EB002E4090009B0107003E40900017
:103F50000080FB00640060000000E000030032000D
:103F600011C0B3002E40900093010700A14A200029
:103F70002E4090000080FB0000004000008F4000B9
:103F80001E007800BE409000014878000080FA00D2
:103F9000000006000800FA0020479800314798000A
:103FA00022079800634798003E4090000004E0001C
:103FB000070032002E4090000080FB00800040008F
:103FC000C080200000804000100F780006003700FD
:103FD0002E4090000080FB00800040008080200088
:103FE00000804000100F78001E0078000000E00004
:103FF00002003A000000EB0037003700AE009000EE
:104000001E007800110098001E007800EE4090001D
:10401000014878001E0078001040900002C4B300F0
:10402000824060001E007800114098001E00780059
:1040300010409000804078000134A0001E007800FD
:10404000114098001E0078001040900080407800D9
:104050000174A0001E007800114098003E409000BE
:104060000004E0000E0032002E4090000080FB00B3
:10407000AE4090008180FB0001814000C1802000A3
:1040800081004100910078000120A2000001400061
:10409000C080200000004100010878000D003700BA
:1040A0002E4090000080FB00AE4090008180FB001D
:1040B0000181400081802000810041009100780052
:1040C0000120A2000001400080802000000041008B
:1040D000010878001E0078000080FA000000060049
:1040E0000400FA0020479800314798002E409000C5
:1040F0000004E00017003A003040800081C0B300A7
:104100000148780030408000A18C20001100980008
:1041100030408000C1C0B3001140980030408000A2
:1041200031408000914090000174A000114098003F
:104130006040800041C0B3001140980060408000A2
:1041400061408000914090000174A00011409800EF
:104150002E0037002E4090000080FB000000400041
:10416000800078003E4090000080FB00008040000E
:104170004300DD008000780000A02000008F400098
:104180001E00780010409000804078000124A000BC
:104190001E007800114098001E007800104090002A
:1041A000804078000174A0001E0078001140980043
:1041B0002E4090000080FB0000004000800078004E
:1041C0003E4090000080FB00008040004300DD0086
:1041D000E400400000A02000008F40001E00780096
:1041E00010409000804078000124A0001E0078005C
:1041F000114098001E007800104090008040780028
:104200000174A0001E007800114098000080FA00A0
:10421000000006000200FA00004F7800A124800090
:1042200000022000008060000000E0005100320029
:104230001E80FB0080004000C08020000080400005
:10424000100278001E80FB0080004000C08020002B
:1042500000804000100078001001BE000004200023
:1042600001002000820278000301780080017800BC
:104270000100780083826200000061008000EB0092
:10428000C000DD00000020000001BE006128B80071
:104290000001710081817100028ABE001E80FB0056
:1042A00080004000C08020000080400010027800A4
:1042B0001E80FB0080004000C08020000080400085
:1042C000100078001001BE00000420000100200052
:1042D0000000690081806900008ABE001E80FB002A
:1042E0009E80FB0001814000C180200081004100D0
:1042F000910078000120A20000014000C080200051
:1043000000004100010878001E80FB008000400092
:10431000C080200000804000900078001E80FB00DC
:1043200000014000C0802000000041001000780023
:10433000104090000044B200904098001E80FB00A6
:1043400080004000C0802000008040009000780085
:104350001E80FB0000014000C080200000004100E2
:10436000100078001041900000C4B30000406900C4
:10437000904098000080FA00000006000000FA005B
:104380009424EF008C24EF000028EF000080FA0056
:10439000000006000000FA00004080000000E0007D
:1043A00014003A009424EF008C24EF002000200039
:1043B00030258800A824EF008644A900F0092000D9
:1043C00080248800F00920006024880082C4A800AE
:1043D0009EC0A800010037009404A800A02480001B
:1043E000610060000000E000FBFF320010002000D0
:1043F000004088000080FA00000006000000FA007B
:104400001BC8BF000004A2000004E000340032001A
:1044100010C0B3001BE8B7001CC8BF000004A20016
:104420000004E0002E00320010C0B3001CE8B7000A
:1044300011C8BF00E24F50000C003A0060408000FD
:104440008040EB00014878006040800081C4B300E8
:1044500011409800604080006140800091409000D1
:104460000174A000114098001D00370011C8BF0062
:10447000E14F50001A003A001868EF002040800019
:1044800081C0B3000148780020408000A18C20004A
:10449000110098002040800041C0B30011409800F6
:1044A0002040800021408000914090000174A000D5
:1044B0001140980010C0B30018E8B70030408000E9
:1044C00081C0B3000148780030408000A18C2000FA
:1044D000110098003040800001C8B30011409800DE
:1044E0000080FA00000006000000FA001D68EF00DE
:1044F0001E68EF0011C8BF00E24F50000F003A00E5
:104500003040800081C0B300014878003040800016
:10451000218D2000110098003040800081C4B3003C
:104520001140980030408000314080009140900060
:104530000174A000114098001D003700008D20007C
:104540001080FB00118D20009180FB00C808DD0069
:104550000100700080007800E0458000808F5000EE
:1045600007003100008D20001080FB00118D20001D
:104570009180FB00C808DD0001007000E045880064
:104580009600070060408000218D200011009800F7
:104590006040800081C4B3001140980060408000FA
:1045A00061408000914090000174A000114098008B
:1045B0000080FA00000006000400FA00204798007E
:1045C0003147980000A02000000F78002E40900096
:1045D0000080FB0000004000800078003E4090001A
:1045E0000080FB00008040004300DD001E0F400003
:1045F0001E0078009000780001F0A100010878000A
:104600003E4090000004E00007003A002E40900079
:104610000080FB008000400080802000008040007F
:104620001E087800060037002E4090000080FB0036
:1046300080004000C0802000008040001E087800FC
:104640001E0078009000780001E0A10001087800C9
:104650009E007800648040009000780001E0A00097
:10466000010878000080FA00000006000000FA004F
:1046700094A4A900D14580000008200000806000BB
:104680000000E00027003A00008C200090407800F5
:1046900000C8B30000C060000004E0000A0032005F
:1046A00020C0B30011E8B7001EC8BF000004A2007C
:1046B0000004E000010032008BFF07001C68EF00DF
:1046C0001B68EF00430037003040800081C0B3001A
:1046D0000148780030408000A18C20001100980033
:1046E00030408000C1C0B3001140980030408000CD
:1046F00031408000914090000174A000114098006A
:104700006040800041C0B3001140980060408000CC
:1047100061408000914090000174A0001140980019
:104720002C003700A08C20009040780000C8B30017
:1047300000C060000004E0000F00320010C0B300B1
:1047400011E8B7001DC8BF000004A2000004E0008B
:104750000100320064FF07001C68EF001B68EF00D7
:104760001AC8BF000004A2000004E00019003200D3
:1047700022FF07001700370020C0B30011E8B70080
:104780003040800081C0B300014878003040800094
:10479000A18C2000110098003040800041C0B3007F
:1047A00011409800304080003140800091409000DE
:1047B0000174A000114098001C68EF001B68EF0016
:1047C0001AC8BF000004A2000004E000010032008B
:1047D0000AFF07000080FA00000006000200FA004D
:1047E00080C0B300004F7800E0458000E70F500024
:1047F0000D003E00E0458000004F780010C8BF006B
:104800000004E00003003A0010C0B30010E8B70055
:104810000500370010C8BF00E14F500002003A0009
:1048200020C0B30010E8B700E14580001E80FB0007
:1048300000805000E0458800604080001E487800FD
:10484000208D200090408800D045800061006000ED
:104850000000E00017003A00090037009140800096
:10486000C045800010417800824878008100E8004F
:10487000914088000000E800C04588001E4FE90014
:104880001E4078000004E000F4FF3A000C003700FE
:1048900091408000C0458000104178008248780037
:1048A0008100E800914088000000E800C0458800D1
:1048B0001E4FE9001E4078000004E000F4FF3A00BB
:1048C0000080FA00000006000200FA00204080008C
:1048D000104F78009E80FB00004680004800DE00FC
:1048E00013468000F20F2000028161004811DD00B4
:1048F00002007000808F50000800360000468000E3
:104900004800DE0012468000F10F200081006100A7
:10491000C808DD0001007000004F780000468000EC
:104920004800DE0012468000F10F20008100610087
:10493000C808DD0001007000800078001E80FB00C8
:1049400000805000F10F200081006000C808DD00E9
:1049500003468000F20F2000028161008280700017
:1049600001468800C800DE00F00F200000806000D3
:104970001246800001F02F008100610001007000EC
:10498000104688000040EB00104798000C003700EC
:10499000F04580009E4090000181FB00218D2000A9
:1049A0008100410091407800014878000000E80053
:1049B000F04588001E4090000040E8001047980035
:1049C0001E4090009E4F5000F1FF390000468000CD
:1049D0004800DE0012468000F10F200081006100D7
:1049E000C808DD00010070000000E0001E00320079
:1049F0003040800081C0B300014878003040800022
:104A0000218D200011009800204080009000780047
:104A100000002400008060000000E00009003A006F
:104A20003040800081C4B3001140980030408000C5
:104A300031408000914090000174A0001140980026
:104A4000300037003040800081C0B3001140980032
:104A50003040800031408000914090000174A000FF
:104A600011409800270037003040800081C0B3001B
:104A70000148780030408000A18C2000110098008F
:104A80003040800041C0B3001140980030408000A9
:104A900031408000914090000174A00011409800C6
:104AA000104680004800DE0022468000F10F200002
:104AB00081006100C808DD00010070000000E00016
:104AC00008003200104680004800DE0022468000C8
:104AD000F10F200081006100C808DD0001007000B6
:104AE00000000100004680000070A1000046880020
:104AF0001AC8BF000004A2000004E0000100320058
:104B00003EFE07000080FA00000006000200FA00E6
:104B1000D04580000070A000D04588002200200011
:104B20008000EB00C04A20003DFB0700020220008D
:104B30008000EB0000A0200039FB07009424A800AF
:104B40000040EB00004F78000B0037009E80FB0018
:104B5000608C2000008040008040EB00014878001D
:104B60009E80FB00808C2000008040008040EB0095
:104B7000014878001E4FE8001E407800E14F5000C9
:104B8000F2FF3600120020008000EB003080200091
:104B900023FB07009424A90080A020006040880027
:104BA00000A0200020408800204080003040880085
:104BB000C08C20001040780002E8B70002C8BF0097
:104BC0000004E00003003A000001200000408800DB
:104BD0000600370012002000218020001000200075
:104BE000BB08070000022000004088000080FA0097
:104BF000000006000000FA00A08C20009040780021
:104C000000C8B30080CF500047003A00A08B2000BE
:104C100001CCB30001487800D08C2000104078000F
:104C20000080FB00E20F500009003200E30F50004B
:104C300023003200E10F500037003A00E0C12900A4
:104C4000C045880020012000E0458800360037007C
:104C5000C08C2000104078000004E00014003A00EE
:104C6000C08C2000104078000080FB000000400055
:104C70008000780060CA29000080400010007800A1
:104C8000C0458800C04580000080E8009040780062
:104C9000C08B200001487800C045800063004000C0
:104CA00090407800D08B2000014878001E0037002B
:104CB000A08B20008040EB00014878001A003700EC
:104CC000C08C200010407800E24F50000E003E00E3
:104CD000C08C2000104078000080FB0000004000E5
:104CE0008000780080CA2900008040001000780011
:104CF000C0458800C0458000104078000080FB005F
:104D0000E045880008003700A08B20008040EB00C1
:104D10000148780004003700A08B20008040EB00A1
:104D200001487800000000000080FA000000060042
:104D30000200FA00208D20008040EB00014878003E
:104D4000308D20008040EB0001487800A08C2000CE
:104D5000904078007FC060000080FB00E10F5000B1
:104D600011003200E20F5000130032000000E0009A
:104D700047003A00D04580000070A000D045880070
:104D800014C8BF000004E0003A003200208D20006B
:104D900010407800804078000114A000208D200091
:104DA000014878003A003700D04580000070A0002C
:104DB000D045880036003700D04580000070A00044
:104DC000D0458800E08C2000104078006F406000E3
:104DD0000004E00029003200E08C200090407800C0
:104DE00000C8B30000C060000004E00009003A0001
:104DF000E08C2000904078006FC060000080FB00D5
:104E0000800040008080200000804000100F78006B
:104E100008003700E08C2000904078006FC06000F0
:104E20000080FB0080004000C08020000080400027
:104E3000100F78001E007800900078000000280015
:104E4000008060000000E0000E0032001E007800CC
:104E50009000780000402000008060000000E0002A
:104E60000A003200208D200011C0B30001487800F4
:104E700007003700000000000500370000000000B8
:104E800003003700000000000100370000000000B0
:104E9000D145800000082000008060000000E00094
:104EA00008003200208D2000C0458800D0458000D9
:104EB0000000A000D0458800C08B200021C0B300B6
:104EC000014878000080FA00000006000000FA00A7
:104ED00050258000620060000000E00013003200F6
:104EE000204080009040900000C8B30080CF500068
:104EF0000D003A00604080009040900040C8B30030
:104F000080CF500008003A0020408000C1C0B300AC
:104F10001140980020408000214080009140900086
:104F20000174A00011409800AA24A90000082000E4
:104F3000502488000080FA00000006000000FA00FB
:104F40008284A800000120005024880010C0B30013
:104F500015E8B7002468EF000001EB008000EB00CB
:104F600050072000DA0707000080FA000000060062
:104F70000000FA001568EF000001EB008000EB0074
:104F800040072000D20707008284A900000120000A
:104F9000002488002468EF000080FA00000006006A
:104FA0000000FA00D0C2B30019E8B70016C8BF006D
:104FB0000080FB000020A1000000E0001F003A007C
:104FC00016C8BF000080FB004200DE0000407800F1
:104FD0000080FB00C200DD0000A020000080400037
:104FE0002040880020408000304088003040800011
:104FF0000020A2003040880020408000900078000F
:1050000000C023008080600000402300808F50009B
:1050100008003A002040800010009000820020002C
:1050200080007800A08C2000F6F907000B00070034
:10503000080037003D0007000600370016C8BF0013
:105040000080FB000020A100E80F500001003A00A2
:10505000530007000080FA00000006000000FA007C
:105060001068EF001A68EF001D68EF001E68EF007F
:105070001868EF001168EF00604080006140800018
:10508000914090000174A1001140980060408000A0
:105090000020A200604088006040800061408000E5
:1050A000914090000174A100114098006040800080
:1050B0000020A20060408800304080003140800025
:1050C000914090000174A10011409800A08B200035
:1050D0008040EB00014878000000EB00E0458800CC
:1050E000008C20008040EB000148780001468000E1
:1050F000F00F20000080600000468800114680000C
:1051000000F02F0000806000104688008300070038
:105110000001EB008000EB00300020006C0707006E
:1051200052FD07000080FA00000006000000FA00AF
:1051300011C8BF00E24F500002003A00E2FD070034
:10514000150037001168EF0018C8BF000004A20066
:105150000004E0000F0032003040800081C0B30046
:105160000148780030408000A18C20001100980098
:1051700030408000C1C0B300114098003040800032
:1051800031408000914090000174A00011409800CF
:10519000010037001868EF000080FA0000000600E8
:1051A0000200FA0060408000100078004E00DE002F
:1051B00061406000004F7800604080000020A20045
:1051C0006040880000408000E80F50000E003A0068
:1051D000C08C2000104078008080FB00F007200089
:1051E00000806000B0248800B02480000000E0004F
:1051F0000300320000012000004088000200370058
:10520000400020000040880011C8BF00E14F50005E
:1052100025003A0060408000218D20001100980098
:105220006EFD070010C8BF00E24F500009003A00B1
:105230006040800041C0B300114098006040800091
:1052400061408000914090000174A00011409800DE
:10525000300037001E4078000004E00009003A00EA
:105260006040800081C4B30011409800604080001D
:1052700061408000914090000174A00011409800AE
:10528000240037006040800081C0B30011409800C6
:105290006040800061408000914090000174A00057
:1052A000114098001B003700008C200090407800CF
:1052B00000C8B30000C060000004E0001400320029
:1052C000104680004800DE0022468000F10F2000DA
:1052D00081006100C808DD00010070000000E000EE
:1052E00008003200104680004800DE0022468000A0
:1052F000F10F200081006100C808DD00010070008E
:1053000000000100004680000070A10000468800F7
:105310001168EF000080FA00000006000000FA00AB
:10532000A08C2000104078000046B2000004E0008D
:1053300051003A00B08C2000104078000080FB0043
:10534000CF80DE00B200200003002000820F50005A
:10535000838F58004A003E000060010021003700A2
:105360002200370048003700200037004600370091
:10537000060037000B0037003A0037000D003700F9
:105380000A0037001B0037002A003700D045800094
:105390000070A000D04588008000200000408800F8
:1053A0003A00370013FE070038003700D7FD07002A
:1053B0003600370020802000C0458800D04580009E
:1053C0000000A000D0458800C08B200011C0B300B1
:1053D00001487800D04580000070A000D0458800CA
:1053E0002A00370052FE0700280037002900070076
:1053F00026003700E08C2000104078008080FB0001
:105400003080200000804000C0458800D0458000EA
:105410000000A000D0458800C08B200011C0B30060
:1054200001487800D04580000070A000D045880079
:1054300016003700D04580000070A000D0458800DD
:10544000E08C2000104078000081FB00C08C200020
:105450009040780030802000000041000148780032
:105460000A0037000001EB008000EB002000200064
:105470009706070005003700000000000300370012
:105480000000000001003700000000000080FA006A
:10549000000006000600FA00C08C200010407800D2
:1054A000E14F500010003A00A08C2000104078001E
:1054B0007F4060000004E0000B003A00D04580000F
:1054C0000070A000D0458800B08C2000104078000B
:1054D000E34F500003003A0010C0B30014E8B700D7
:1054E000010037001468EF00C08C200010407800E5
:1054F0000004E000F7003A00A08C20001040780083
:105500007F406000E24F5000F2003A00E08C200043
:10551000104078006F4060000004E000ED003200B1
:10552000E08C2000904078006FC060000080FB009D
:10553000E10F5000E7003C00014080000002200025
:10554000808F5000E3003A00D04580000070A0003A
:10555000D0458800E08C20009040780000C8B3005F
:1055600000C060000004E00011003A00E08C200060
:10557000104178006F4061000080FB008000400017
:105580008080200000804000100F7800E08C200018
:10559000904078006FC060008080FB00808C20000D
:1055A000008040001040780040479800100037000D
:1055B000E08C2000104178006F4061000080FB000B
:1055C00080004000C080200000804000100F780064
:1055D000E08C2000904078006FC060008080FB006D
:1055E000608C200000804000104078004047980008
:1055F0004E409000614060000004E00004003A006A
:105600001E0078000020A100000F78000300370082
:105610001E0078000020A000000F7800E08C200021
:105620009040780000C8B30000C060000004E000B3
:105630000A003A00E08C2000104178006F406100C1
:105640000080FB009E007800000140008080200068
:10565000000041000108780009003700E08C2000BC
:10566000904078006FC060000080FB009E007800D2
:1056700000014000C08020000000410001087800C7
:10568000B08C200010407800E34F50002C003A000E
:105690001E00780090007800000028000080600064
:1056A0000000E00019003200E08C200090407800FB
:1056B00000C8B30000C060000004E0000A003A0027
:1056C000E08C2000104178006F4061008080FB007A
:1056D000808C200000804000904078000114A000E1
:1056E0000148780009003700E08C200090407800E5
:1056F0006FC060008080FB00608C20000080400054
:10570000904078000114A000014878001E00780045
:1057100010409000804078000124A0001E00780016
:10572000114098001E0078001040900080407800E2
:105730000174A0001E007800114098006500370039
:105740001E0078000020A200000F78001E007800E4
:105750009000780000002800008060000000E00059
:10576000110032001E007800104090008040780048
:105770000174A1001E007800114098001E007800FE
:1057800010409000804078000164A0001E00780066
:1057900011409800220020009E0078005000200058
:1057A000CB050700060037001E007800104090006F
:1057B000804078000164A0001E007800114098002D
:1057C0001E0078000020A200000F78004E409000DC
:1057D000624060000004E00006003A001E0078000D
:1057E0009000780000002800008060000000E000C9
:1057F00024003200E08C20009040780000C8B30004
:1058000000C060000004E0000A003A00E08C2000C4
:10581000104178006F4061008080FB00808C200088
:1058200000804000904078000114A10001487800F9
:1058300009003700E08C2000904078006FC06000C5
:105840008080FB00608C2000008040009040780049
:105850000114A100014878001E007800104090005B
:10586000B2C3B300824060001E007800114098006F
:10587000220020009E0078005000200094050700C0
:10588000060037001E00780010409000B2C3B3003D
:10589000824060001E00780011409800A14A20005C
:1058A000E08C2000104178006F4061000080FB0018
:1058B0000000400000804000100798001E0090008B
:1058C00010407800804078000114A1001E00900074
:1058D000014878000080FA00000006000000FA008D
:1058E000004180001141800061004000E0804800DC
:1058F000004188001141880015C8BF000004A200C3
:105900000004E0000800320024C8BF000040E800A6
:1059100024E8B70024C8BF000004E00002003A00F9
:1059200000C0EB0024E8B7000080FA000000060089
:105930000400FA000241800013418000028FBE0083
:1059400000418000114180001E01BE00800F510007
:10595000818F5900F7FF3A001E00BE000080FA0058
:10596000000006000200FA00000F78001E00780018
:10597000E40F500018003200E40F500007003E0012
:10598000E20F500010003200E20F500010003E0005
:10599000E10F50000A00320019003700E60F5000F6
:1059A00011003200E60F50000D003900E70F5000E3
:1059B0000F003200E80F50000F00320010003700D7
:1059C000F4C2A8000E003700DDE2A8000C0037008A
:1059D000F502A8000A003700F522A80008003700E9
:1059E000F4C2A80006003700F4C2A8000400370083
:1059F000F4C2A80002003700F4C2A80000000000B2
:105A00000080FA00000006000200FA00000F780093
:105A10001E007800E40F500018003200E40F500020
:105A200007003E00E20F500010003200E20F50006D
:105A300010003E00E10F50000A003200190037004C
:105A4000E60F500011003200E60F50000D00390043
:105A5000E70F50000F003200E80F50000F00320037
:105A600010003700F4C2A9000E003700DDE2A900E3
:105A70000C003700F502A9000A003700F522A90042
:105A800008003700F4C2A90006003700F4C2A900DC
:105A900004003700F4C2A90002003700F4C2A900D4
:105AA000000000000080FA00000006000200FA007A
:105AB000000F78001E007800E40F5000380032001C
:105AC000E40F500007003E00E20F50001B003200C0
:105AD000E20F500025003E00E10F50000A003200A6
:105AE00070003700E60F500047003200E60F50000C
:105AF00038003900E70F500050003200E80F500026
:105B00005B00320067003700A01780004600DE000F
:105B1000614060000004A200614060000080FB0062
:105B2000610060004600DD00A11780000160A10057
:105B300001007000A01788005A003700E0168000AE
:105B40004F00DE00004078000004A20061406000C9
:105B50000080FB004F00DD00E116800001F0A10095
:105B600001007000E01688004E003700A01780008A
:105B70004800DE00614060000004A2006140600057
:105B80000080FB00610060004800DD00A11780007C
:105B90000180A10001007000A017880041003700BB
:105BA000A01780004900DE00614060000004A200F0
:105BB000614060000080FB00610060004900DD0082
:105BC000A11780000190A10001007000A0178800BB
:105BD00034003700A01780004600DE0061406000FE
:105BE0000004A200614060000080FB0061006000D2
:105BF0004600DD00A11780000160A10001007000D7
:105C0000A017880027003700A01780004600DE009C
:105C1000614060000004A200614060000080FB0061
:105C2000610060004600DD00A11780000160A10056
:105C300001007000A01788001A003700A01780002C
:105C40004600DE00614060000004A2006140600088
:105C50000080FB00610060004600DD00A1178000AD
:105C60000160A10001007000A01788000D0037003E
:105C7000A01780004600DE00614060000004A20022
:105C8000614060000080FB00610060004600DD00B4
:105C9000A11780000160A10001007000A01788001A
:105CA000000000000080FA00000006000200FA0078
:105CB000000F78001E007800E40F50002D00320025
:105CC000E40F500007003E00E20F500017003200C2
:105CD000E20F50001E003E00E10F50000A003200AB
:105CE00051003700E60F500034003200E60F50003C
:105CF00029003900E70F500039003200E80F50004A
:105D00004000320048003700A11780000004200046
:105D10000080600000F0A7000000EA000000EA0038
:105D20004F00DE000040780040003700E1168000A0
:105D3000000028000080600000F0A7000000EA00DA
:105D40000000EA004F00DE00004078003700370016
:105D5000A1178000001020000080600000F0A70064
:105D60000000EA000000EA004F00DE00004078007A
:105D70002E003700A1178000002020000080600066
:105D800000F0A7000000EA000000EA004F00DE007B
:105D90000040780025003700A11780000004200093
:105DA0000080600000F0A7000000EA000000EA00A8
:105DB0004F00DE00004078001C003700A117800073
:105DC000000420000080600000F0A7000000EA004E
:105DD0000000EA004F00DE000040780013003700AA
:105DE000A1178000000420000080600000F0A700E0
:105DF0000000EA000000EA004F00DE0000407800EA
:105E00000A003700A1178000000420000080600015
:105E100000F0A7000000EA000000EA004F00DE00EA
:105E200000407800010037000040EB000080FA00DD
:105E3000000006000200FA00000F78001E00780043
:105E4000E40F500018003200E40F500007003E003D
:105E5000E20F500010003200E20F500010003E0030
:105E6000E10F50000A00320019003700E60F500021
:105E700011003200E60F50000D003900E70F50000E
:105E80000F003200E80F50000F0032001000370002
:105E9000F0C2A9000E003700D9E2A9000C003700BB
:105EA000F102A9000A003700F122A900080037001A
:105EB000F0C2A90006003700F0C2A90004003700B4
:105EC000F0C2A90002003700F0C2A90000000000E3
:105ED0000080FA00000006000000FA00A60007009B
:105EE00014C8BF000004E0000100320015C8BF0064
:105EF0000040FE005124800000022000008060006D
:105F00000000E00002003A0010C0B30041000700AA
:105F1000D200070010C0B3000080FA0000000600A5
:105F20000000FA0014C8BF000004E0003600320090
:105F300015C8BF000004E000330032004024800098
:105F4000620060000000E000010032008824A90027
:105F500075000700000420000024880000000000F5
:105F60000124800000042000008060000000E000A8
:105F7000FBFF320000042000002488000000000025
:105F80000124800000042000008060000000E00088
:105F9000FBFF320000042000002488000000000005
:105FA0000124800000042000008060000000E00068
:105FB000FBFF32009444A800000420000024880065
:105FC0000000000001248000000420000080600028
:105FD0000000E000FBFF32000004200000248800E5
:105FE0000000000001248000000420000080600008
:105FF0000000E000FBFF32009444A90057000700B6
:1060000010C0B300010037000040EB000080FA0030
:10601000000006000400FA00204798004024800099
:10602000610060000000E0000B00320040248000AE
:10603000620060000000E00007003A0024C8BF00D2
:10604000E34F500004003600202480004300DE00AF
:1060500061406000320037002E4090000004E000F4
:106060001D0032008824A9008804A8002E00070023
:106070000040EB00004F78000900370000042000CA
:10608000002488000000000001248000000420009B
:10609000008060000000E000FBFF32001E4FE800BF
:1060A0001E407800E44F5000F4FF36000040EB0043
:1060B0001047980020248000680060000000E00085
:1060C0000200320010C0B300104798002300070000
:1060D0001E409000120037004024800061006000E4
:1060E0000000E00002003A0000C0EB000C003700A6
:1060F00040248000620060000000E00002003A00DE
:10610000E0CFB3000600370024C8BF00E34F5000C3
:1061100002003E00D0CFB30001003700C0CFB30073
:106120000080FA00000006000000FA002E68EF0070
:106130001000FC00F10480000004200000806000DA
:106140000000E0000200320010C0B3002EE8B700EB
:106150009EC0A9000080FA00000006000000FA00BE
:106160002EC8BF000004E000010032009EC0A8005D
:106170000080FA00000006000400FA001E00FC0087
:1061800011028000000E2000008060003041880075
:1061900011028000000E2000010070001002880033
:1061A00040092000100798000000EB00000F780065
:1061B0000E0037001E009000900078001E0078004E
:1061C00000014000A08D200000004100010878007F
:1061D0001E0090008000EB00010878001E00900077
:1061E0000080E800100798001E0FE8001E007800ED
:1061F000E50F5000EFFF360060248000404188002A
:106200008C24EF0010248000504188008224EF008D
:10621000700680004800DE00674060000080FB00E0
:106220006041880000012000002488000002200056
:10623000502488008EC0A9008284A80071068000C6
:10624000F08F2F000080600000A0A0007006880082
:106250009EC0A8000080FA00000006000400FA00BA
:1062600040092000100798000000EB00000F7800A4
:106270000B0037001E00780080004000A08D200039
:1062800000804000900078001E0090000108780017
:106290001E0090000080E800100798001E0FE80024
:1062A0001E007800E50F5000F2FF360040418000EC
:1062B00060248800504180001024880060418000E4
:1062C00000407800674060000080FB0067006000CD
:1062D0004800DD0072068000F18F2F008100610010
:1062E000010070007006880011028000F0F12F009C
:1062F00080806000304180000100700030418800E3
:1063000030418000100288000080FA000000060082
:106310000000FA000117800000F02F0000806000EC
:1063200000178800F002A900F022A900E822A900C5
:10633000F402A900F422A900EC22A90000502300D5
:10634000C1002000580307008040EB0080C3B30069
:10635000110007008040EB0080C0B3000E00070072
:106360008040EB0010C0B3000B0007008040EB0042
:1063700060C0B300080007008040EB00C0C0B3005D
:106380000500070000B82B000100200046030700AD
:106390000080FA00000006000400FA002047980080
:1063A0003147980001178000F00F200001007000B5
:1063B00000178800F422A800F402A9002117800029
:1063C00000F02F000080600020178800EC22A80059
:1063D0000000000000000000000000001017800016
:1063E0004700DE0061406000004F7800EC22A90009
:1063F0001E4078000004E000F4FF3A00011780001E
:1064000000F02F000080600000178800F422A9002F
:106410003E4090000080FB000000EA004F00DE00DC
:10642000004078000080FB0061006000A117800040
:106430000100A10001007000A01788002117800052
:1064400000F02F00808060002E4090000080FB0054
:106450000100700020178800EC22A8000000000056
:106460000000000000000000EC22A9000080FA00FB
:10647000000006000400FA00100798008F003700A3
:106480001E009000104F78001E00FB006101B90053
:106490000005200001002000020040008380480029
:1064A000C204200003002000820F5000838F580098
:1064B00075003E0000600100700037007200370078
:1064C00071003700700037006F0037006800370038
:1064D0006D0037006C0037006B0037006A00370032
:1064E0006900370068003700670037006600370032
:1064F0006500370064003700630037006200370032
:1065000061003700600037005F0037005E00370031
:106510005D0037005C0037005B0037005A00370031
:106520005900370058003700570037005600370031
:106530005500370054003700530037005200370031
:1065400051003700500037004F0037004E00370031
:106550004D0037004C0037004B0037004A00370031
:106560004900370048003700470037004600370031
:106570004500370038003700430037001B00370064
:1065800041003700400037003F0037003E00370031
:106590003D0037003C0037003B0037001600370055
:1065A0003900370038003700370037001500370052
:1065B00035003700340037002A003700320037003A
:1065C00031003700120037002F0037001C00370061
:1065D0001E0037002C0037002B0037002A00370040
:1065E0000E003700130037000F0037000040EB00AB
:1065F000004F78002400370010C0B300004F78002F
:106600002100370020C0B300004F78001E00370083
:1066100030C0B300004F78001B00370040C0B3000B
:10662000004F78001800370050C0B300004F7800CA
:106630001500370060C0B300004F7800120037002B
:1066400070C0B300004F78000F003700F0CEB300E9
:10665000004F78000C00370080C0B300004F780076
:106660000900370090C0B300004F780006003700E3
:1066700040CEB300004F780003003700F0CDB300E8
:10668000004F7800000000001E407800EA4F5000E4
:1066900004003A008040EB0000CCB3003EFF07004E
:1066A000030037001E40780011C0B3003AFF070016
:1066B0001E0090000000E800100798001E009000E7
:1066C000104078000004E0006DFF3A000080FA00FE
:1066D000000006000200FA008040EB0000C4B30096
:1066E0002DFF07000000EB00000F780006003700C8
:1066F000E0CA29001E0040001040780011C0B3001D
:1067000025FF07001E0FE800F00420009E0078001F
:10671000808F5000F6FF34008040EB0000C8B300CB
:106720001DFF07000080FA00000006000000FA00CC
:106730003228EF00D1C1B30010C0B300F8F5070054
:1067400003C4B300828320008040EB0010C0B3007C
:1067500010F60700804188000080FA000000060063
:106760000200FA0000408000FF0F50006500360074
:1067700040248000620060000000E00063003A00F6
:10678000804180000000E00006003200804180006F
:106790009000780000002800008060000000E00009
:1067A0005B003A0080832000104078000080FB00EE
:1067B00001082000810F500007003200110820005E
:1067C000810F50000700320071032000810F50003C
:1067D000230032004400370020002000B3FC0700F3
:1067E00041003700904180000000E00006003200C8
:1067F0009041800090007800000028000080600038
:106800000000E00035003A008087200011C8B30086
:106810000148780010002000260107000004A200B3
:106820000004E000040032009087200011C0B30093
:106830000148780003003700908720008040EB007B
:106840000148780003C4B3008287200011C0B30060
:1068500010C0B300CFF50700904188002200370038
:10686000904180000000E00006003200904180006E
:106870009000780000002800008060000000E00028
:1068800018003A00400020003E000700000F78008A
:106890008087200071C3B300014878001E00780093
:1068A0008040780090872000014878001E00780022
:1068B0004800DE0080407800A08720000148780072
:1068C00003C4B3008287200011C0B30010C0B3001E
:1068D000B0F5070090418800030037000000000079
:1068E000010037000000000003C4B30082832000D1
:1068F0008040EB0010C0B300A6F50700804188007F
:106900000300370000000000010037000000000015
:106910000080FA00000006000400FA00100798004A
:106920001E009000E40F500004003200E50F5000FC
:106930000400320000C0EB0010003700000000002F
:1069400001003700000000001E0090000D0007004D
:10695000D1CC2C000100B8004308DE00004F7800C5
:1069600040C6B3009E40780080CF50000200360041
:1069700040C6B300004F78001E4078000080FA0047
:10698000000006000400FA00100798001E009000A6
:10699000E40F500004003200E50F50000400320004
:1069A0000080EB001F0037000000000001003700EE
:1069B000000000009E009000411988002023A800DC
:1069C0000000EB00000F780002003700000000001C
:1069D0001E0FE800703E20009E007800808F50005F
:1069E000FAFF36002023A9000000EB00000F78001A
:1069F00002003700000000001E0FE800703E20007B
:106A00009E007800808F5000FAFF360000000000E2
:106A100000198000610060000000E000FCFF32000F
:106A2000001880000080FA00000006000200FA0052
:106A3000000F78001E007800E40F500005003200BF
:106A4000E50F500006003A002CA3A90010C0B300C7
:106A5000040037002C83A90010C0B30001003700E8
:106A60000040EB000080FA00000006000200FA007F
:106A7000000F78001E0078000000E0001A003A00C5
:106A800011198000F0FF21000080600010198800BB
:106A900040C0B30024E3B70001198000F0F12F00DB
:106AA000008060000019880021198000F00F2E007E
:106AB0000080600000C0A00020198800011980003B
:106AC000F0CF2F00008060000019880011198000AD
:106AD00030FC2F00008060001019880021E3A8001E
:106AE00010C0B300010037000040EB000080FA0046
:106AF000000006000000FA00A08C20001040780082
:106B00007F406000E14F500061003A00E08C2000BF
:106B1000104078000004E0005F003A00B08C2000D4
:106B200010407800E64F500022003A00D08C200040
:106B3000104078000080FB0021022000810F5000EF
:106B40001100320031022000810F50001600320087
:106B500011022000810F500016003A0002C8BF0049
:106B6000E14F500012003A0020C42900C0458800BF
:106B700090002000E0458800A08B200001CCB300ED
:106B8000014878000B00370080C82900C045880004
:106B9000D0012000E0458800A08B200001CCB3008C
:106BA00001487800030037000000000001003700B2
:106BB00000000000A08C20001040780002C6B30046
:106BC0008240600000C2B30080CF500034003A0021
:106BD000B08C2000104078000080FB00E30F5000D4
:106BE0001B003200E30F500005003C00E10F500095
:106BF0002D003200E20F5000060032002B0037005B
:106C0000EA0F50000B003200EB0F5000180032006A
:106C10002600370040832000C04588001000200077
:106C2000E0458800A08B200011CCB300014878001B
:106C30001E003700A08B200001C8B3000148780077
:106C4000D08C20001040780034E8B70017003700DF
:106C500050832000C045880010002000E0458800D7
:106C6000A08B200011C8B300014878000F00370046
:106C7000A08B200001C8B30001487800C08C200020
:106C80001040780035E8B70000000000070037002A
:106C9000000000000500370000000000030037007E
:106CA0000000000001003700000000000080FA0032
:106CB000000006000200FA00000F78001E007800B5
:106CC000E20F500012003200E20F500003003E00BD
:106CD000E10F50000600320027003700E30F50009C
:106CE00014003200E40F50001B0032002200370075
:106CF000901680006200600000F0A7000000EA002B
:106D00000000E9004F00DE00004078001B00370063
:106D100011178000002020000080600000F0A70014
:106D20000000EA000000E9004F00DE0000407800AB
:106D30001200370011178000001020000080600052
:106D400000F0A7000000EA000000E9004F00DE00AC
:106D5000004078000900370090168000680060004D
:106D600000F0A7000000EA000000E9004F00DE008C
:106D700000407800010037000040EB000080FA007E
:106D8000000006000200FA00000F78001E007800E4
:106D9000E20F50000C003200E20F500003003E00F2
:106DA000E10F5000060032000D003700E30F5000E5
:106DB00007003200E40F50000700320008003700DF
:106DC000D022A80006003700E122A8000400370006
:106DD000E102A80002003700D062A8000000000015
:106DE0000080FA00000006000000FA004024800045
:106DF000620060000000E00003003200100020008C
:106E000001FB070030003700014080000002200035
:106E1000808F500013003A00B0418000E10F500015
:106E200003003A0010002000CEFA070023003700CC
:106E3000B1418000B0042000808F500003003A0070
:106E400010002000F0FA07001C003700B14180005C
:106E500060092000808F5000150036003628EF00B2
:106E600016003700B0418000E10F500003003A00E7
:106E700010002000BBFA070010003700B14180006D
:106E800020032000808F500003003A0010002000F3
:106E9000DDFA070009003700B1418000603B2000A7
:106EA000808F5000040036003628EF0003003700C2
:106EB000000000000100370000000000B041800029
:106EC0000000E800B04188000080FA0000000600E1
:106ED0000600FA00000F78001107980022079800BA
:106EE0001E00780021072000810F5000250032008D
:106EF00021072000810F50000A003C00E20F5000E3
:106F000022003200E20F500003003C00E10F50006D
:106F1000180032001E003700E30F50001700320047
:106F20001B00370041072000810F50000D00320088
:106F300041072000810F5000040035005107200058
:106F4000810F50000300320011003700A6FF070038
:106F50000F003700A4FF0700100020002B000700DF
:106F60000B003700A0FF07002000200027000700CB
:106F700007003700EDFD070005003700DDFE0700C4
:106F8000030037000000000001003700000000008F
:106F900010C0B3000080FA0000000600B80800002E
:106FA0002200000000000000000800002600000091
:106FB00000000000000A00002000000000000000A7
:106FC000DA0800000C0000000000000026080000A5
:106FD0000A00000000000000340800000200000069
:106FE0000000000036080000020000000000000061
:106FF0003808000080000000000000003008000099
:107000000400000000000000000000000200FA0080
:10701000000F78001E007800E10F50000F003200D2
:10702000E10F50000F0031001000200081FB07002D
:10703000200020007FFB07001000200051FF070008
:10704000CDE2A900C9E2A9000000EB0087FE07001D
:107050004000200075FE0700030037009EFB07007C
:1070600001003700000000000080FA000000060068
:107070000000FA000000EB00E4FF07006BF20700DD
:10708000C4F40700A2FC070092FD07008040EB005B
:1070900010C0B300C0FC070060D02900F5FC070059
:1070A000AFFD0700FEFF3700F03FB1000180B100E7
:1070B00006003500EE03090000000000403FB1006B
:1070C0000180B100FBFF3D001000B000203FB00088
:1070D00002003500008009000000000000000600EA
:020000040001F9
:020000040002F8
:020000040003F7
:020000040004F6
:020000040005F5
:1057F000FFFF0000FFFF0000B62300007F3E000017
:00000001FF
